:020000040000FA
:100000000128831619308500FF3086008312851081
:10001000051100005420A2201620542005190B2899
:10002000A2203520542085181028092800008618A1
:100030001B28061E051506182128061E0515861EF6
:100040000515051A2928061E0515861E0515061F05
:10005000051585193328061E0515861E0515061F6C
:100060000515861F0515000008000000051A3A282E
:10007000051C851406184028861F8514051C851448
:1000800086184828061F8514861F8514051C8514AC
:1000900006195228861E8514061F8514861F85148E
:1000A000051C8514000008000000061A5D28831650
:1000B0000612861683120612E520861A6628831613
:1000C00086120616061783128612E520061B6F2875
:1000D000831606138616861783120613E520861BE1
:1000E0007828831686130617051483128613E520D5
:1000F0000518802883160510861783120510E52041
:100100000000061987288316061183120611861827
:100110008D2883168610831286100618932883165E
:10012000061083120610051A9928831605128312E9
:10013000051285199F2883168511831285110000E9
:10014000E520080000000619AD28061AAD28831620
:100150000615831285100511D7208618B728861A30
:10016000B72883168614831285100511D720061828
:10017000C128061BC1288316061483128510051199
:10018000D720051ACB28861BCB2883160516831289
:1001900085100511D7208519D5280518D52883166F
:1001A0008515831285100511D720000008005030F6
:1001B0008C00542030308D00FF308E008E0BDE28F6
:1001C0008D0BDC288C0BD9280800FF308F008F0B9B
:0401D000E728080014
:02400E00F13F80
:00000001FF
